:020000040000FA
:02000000FE29D7
:08000800A000030E8312A10009
:100010002608820020342034203420342034203438
:100020006534733463342E34613473346D34203466
:10003000563431342E3435342034203420342034B6
:100040004534533443344334203420342034203472
:10005000B801B901BA01B90AB601B7010310B50D6B
:10006000B80D03183628B90DBA0D2E28B80CB50CEA
:100070003508B3023808031C013EB402031C4C28A7
:100080003908B6043A08B7040310BA0CB90C0318BF
:100090000800B80CB50C38283508B3070318B40AA3
:1000A0003808B4074428B601B7013508B800381C31
:1000B0005F283308B60734080318013EB70703105A
:1000C000B80C3808031908000310B30DB40D5728F5
:0C00D000263E8200663E8200A63E8200B2
:1002000085010000FB2927088500FD21FD21FD2136
:10021000FD2100008501FB2927088500F929000040
:100220008501122927088500F92900008501182970
:100230001129000085011C291729000085012029AA
:1002400000001B290000850125291F2900340334E3
:10025000E634E634E634E634E634E634E634E634CE
:10026000E634E634E634E634E634E634E634E634BE
:10027000E634E634E634E634E634E634E634E634AE
:10028000E634E634E634E634E634E634E634E6349E
:10029000E634E634E634E634E634E634E634E6348E
:1002A000E634E634E634E634E634E634E634E6347E
:1002B000E634E634E634E634E634E634E634E6346E
:1002C00022341D34193415340F340C340034003406
:1002D000FB34F734F334F034EC34E934E634E2340C
:1002E000DF34DB34D734D434D034CC34C834C434E1
:1002F000C034BB34B634B234AD34A734A2349C34E9
:1003000096349034893482347B3473346A34613463
:1003100058344E34433437342A341D340E340934BF
:1003200009340934093409340934093409340934E5
:1003300009340934093409340934093409340934D5
:100340000834083408340834083408340834C8340D
:10035000C934C934C934C934C934C934C934C934B5
:10036000C934C934C934C934C934C934C934C934A5
:10037000C934C934C934C934C934C934C934C93495
:10038000C934C934C934C934C934C934C934C93485
:10039000C934C934C934C934C934C934C934CC3472
:1003A000CF34D334D734DA34DD34E134E434E734D1
:1003B000EA34EC34EF34F234F434F734F934FC3406
:1003C000003400340034003400340034A218ED2925
:1003D000A214000085012908F229270885002808B1
:1003E000A210000081000B11210E8300A00E200E30
:1003F00009002808F2292908F22908008316FF239A
:100400009000831201308A00850183163030013854
:100410009F001030950000308100DF30FB398500EF
:100420008312FF3081008B1601309F00A20114302F
:10043000A300A501A701A801A901E630A600FF308D
:10044000AF00B000B100B2008B17E5222218252AB8
:100450004308BC00BE004208BB00403EBD0003187C
:10046000BE0AE5222218312A42083D024308031C35
:10047000013E3E020318312A4208BD004308BE0077
:100480003B083D02B300AD003C08031C013E3E02A8
:10049000B400AE004030B50028203608AC00B300F0
:1004A000B40153203608AD023708031C013EAE02EA
:1004B0000310AE0CAD0C3B08AD073C080318013E21
:1004C000AE07E5222218612A3D0842023E08031CBD
:1004D000013E430203183C2A4208B3004308B4001B
:1004E00010230038031D612A8B17CB22D822CB2280
:1004F0008B17A501A701BB222308A40009232218FA
:100500007C2A6820003C031D7C2AA40B7E2A013033
:10051000A300A7018501A501BB222030A700092364
:100520002218792A25020319A12A03189B2AA50A51
:10053000BB2222118F2A221D9F2AA502BB2222152F
:100540008F2A22112608003C031D8F2A851D8F2A21
:100550000430A7000130A500BB2209232218792A04
:100560006820003C031D892A250A3F3C031CAD2A54
:10057000A50ABB22AD2A25086A20AA0025086C20FE
:10058000AB00250868208B12A6002A08A8002B08BB
:10059000A9008B160800C830BF0020308500FD215F
:1005A000FD21FD21FD218501DE22BF0BCD2A0800A2
:1005B000C830BF00DE22BF0BDA2A080064003230E8
:1005C000C000FD21C00BE12A0800242322180800E6
:1005D0000530C1000E08C2000F08C30024232218F2
:1005E00008004208FD3EB3004308031CFF3EB40070
:1005F00033080E02B3003408031C013E0F02B4009E
:10060000031DE52A073033020318E52AC10BEE2A41
:1006100008002423221800340E08B3000F08B40089
:100620002D08B3022E08031C013EB402031C003443
:100630002C08B5002820B708031D3F34403036028F
:1006400003183F343608080022104030C4001B3025
:10065000C5008E018F0141309000512322180034D3
:100660000E080F0403192D2B03309F00512322186D
:10067000003409300F0203184B2B051E362B900156
:100680009F18562B5823553C0318562B03300F0246
:10069000031C292B0800512322180034051E4B2B64
:1006A000292B6400C40B0800C50B080022140800A5
:1006B0003108B2003008B1002F08B0001E08AF00AA
:1006C000C600C7013008C6070318C70A3108C607A5
:1006D0000318C70A3208C6070318C70AC70CC60C96
:0806E000C70CC60C4608080017
:02400E00CC3FA5
:00000001FF
